S123F8003838380102060C1080000C0603060C000000060C180C060000001B1B1B1B1B00AD
S123F8200000080C0E0C08000000001F0E040000000000040E1F0000000012161E161200BE
S123F8400000090D0F0D0900002A204C434420546573742E2E2E20202020202020202020C2
S123F860202020202020202020202020202020202A00010203040506078601B7103D8633FA
S123F880B71039861FB7103586FFB7100701BDF8A820FE18CE1800368655B7103A86AAB7FD
S123F8A0103A32180926FC39CEF800A600BDF904BDF893088CF80926F28640BDF904BDF8FC
S123F8C093A600BDF8FCBDF893088CF84926F28680BDF904BDF893A600BDF8FCBDF8930856
S123F8E08CF87126F286C0BDF904BDF893A600BDF8FCBDF893088CF87926F23936B61003BB
S123F9008A04200636B6100384FBB7100332B71004B610038A08B7100384F7B71003393B0C
S123FFD6F91FF91FF91FF91FF91FF91FF91FF91FF91FF91FF91FF91FF91FF91FF91FF91F87
S10DFFF6F91FF879F879F879F87921
S9030000FC
